:03000000023408BF
:0C34080078FFE4F6D8FD75816C02344FAB
:100F5E0020000A3C2E2E2E3E004950436F6E6E65C9
:100F6E0063745245510A004950436F6E6E65637447
:100F7E00000A49504E6F41434B210A003E432C5606
:100F8E002C43432CC0E4E0EFF2E5F020D1E8EDEA8B
:100F9E00EEEC49500A003E432C4D41432C25303295
:100FAE0062583A25303262583A25303262583A2524
:100FBE00303262583A25303262583A253032625811
:100FCE002C4D414320E0E4F0E5F10A003E432C565F
:100FDE0045522C20332E3220EEF22025732025731D
:100FEE002CC2E5F0F1E8FF20495020ECEEE4F3EBE3
:100FFE00FF0A004175672032302032303134003123
:10100E00373A35373A3130003E432C4C442C50524F
:10101E004F473A2020202020202020202020202052
:10102E0020202020202020202020202020202020B2
:10103E0020202020202020202020202020202020A2
:10104E002020202020202020202020202020202092
:10105E0020202020202020202CC4E0F2E020EFF0E1
:10106E00EEF8E8E2EAE828F4E0E9EB290A003E2A85
:10107E002C312CCEF1EDEEE2EDFBE520EFE0F0E0D1
:10108E00ECE5F2F0FB20F1E5F2E5E2EEE3EE20E82E
:10109E00EDF2E5F0F4E5E9F1E00A003E412C4130D5
:1010AE00312C2562752E2562752E2562752E2562D0
:1010BE00752C495020E0E4F0E5F120E0E4E0EFF299
:1010CE00E5F0E00A003E412C4130342C2562752EAD
:1010DE002562752E2562752E2562752CCCE0F1EAFF
:1010EE00E020F1E5F2E80A003E412C4130352C2596
:1010FE0062752E2562752E2562752E2562752CD889
:10110E00EBFEE70A003E2A2C312CCFE0F0E0ECE5B6
:10111E00F2F0FB20EEE1ECE5EDE020EFEE20EFF05B
:10112E00EEF2EEEAEEEBF3205544503937320A0078
:10113E003E412C4130322C2562752E2562752E25AE
:10114E0062752E2562752C495020E0E4F0E5F12001
:10115E00EEF1ED2E20F1E5F0E2E5F0E00A003E4181
:10116E002C4130332C2562752E2562752E25627525
:10117E002E2562752C495020E0E4F0E5F120F0E5D3
:10118E00E72E20F1E5F0E2E5F0E00A003E422C53B6
:10119E0030322C2562752CCEE1ECE5ED20F120F1FC
:1011AE00E5F0E2E5F0EEEC20E1E5E720EAE2E8F238
:1011BE00E0EDF6E8E90A003E422C5330332C25626E
:1011CE00752CCFE5F0E5E7E0EFF3F1EA20EFF0E87C
:1011DE0020EFEEF2E5F0E520F1E2FFE7E820F12066
:1011EE00F1E5F0E2E5F0EEEC0A003E422C53303829
:1011FE002C2562752CCCE5E4EBE5EDEDFBE9204901
:10120E005020EAE0EDE0EB28E7E0E4E5F0E6EAE086
:10121E0020E4EE203520F1E5EA290A003E454E4451
:10122E000A000A44756D705820202020203030208E
:10123E0030312030322030332030342030352030E1
:10124E00362030372030382030392030412030429F
:10125E00203043203044203045203046000A3A00EA
:10126E003A20000A000A44756D7044202020202088
:10127E0030302030312030322030332030342030A6
:10128E00352030362030372030382030392030416C
:10129E00203042203043203044203045203046005C
:1012AE00457272206B657900526420656570726FAD
:1012BE006D0A005264204D454D0A00526420436F62
:1012CE0064650A00577269746520436F64650A008D
:1012DE0044656275674950204F4E0A004465627539
:1012EE00674950204F46460A00446562756755733C
:1012FE006572204F6E0A004465627567557365729C
:10130E00204F46460A0044656275674D7367204F4D
:10131E006E0A0044656275674D7367204F46460A34
:10132E0000436F6E666967206C6F636B210A00570E
:10133E007220656570726F6D0A00205361766520AC
:10134E00656570726F6D210A00457272204D4143C2
:10135E0021004C6F61643E3E002A00CEF8E8E1EABF
:10136E00E00A00202D202575282575290A003C410C
:10137E0030313D003C4130323D003C4130333D0088
:10138E003C4130343D003C4130353D003C21003C79
:10139E005330323D003C5330333D003C5330353DED
:0D13AE00003C5330383D003C5330363D00CC
:063D560001690001670095
:103DBC00C28E438910E4F58B758DB8D2ABD28E22AE
:0A3DDB00E4FEEEC39F50030E80F8D3
:013DE50022BB
:03001B0002337835
:10337800C0E0C083C082C0D0C28E758B00758DB886
:10338800201E0675A61E75A6E10567D21AE56960B6
:10339800020569056CE56C540F7051E568D394011A
:1033A80040021568D226E56C543F7012D218906618
:1033B8008EE0600A04F0E0D394B44002D21E906616
:1033C80087E0600204F0906104E0600214F0906607
:1033D8008FE0D394014003E014F0301D02056AE544
:1033E8006BD394644004D21E8002056BE566D394C7
:1033F8000140021566D28ED0D0D082D083D0E03280
:1008E000C291C290D2B5C2237D027C007F07123D27
:1008F000398F27E527646060097D017F60123CB66F
:10090000D223E4FDFC7F0B123D398F27E52730E62B
:10091000097D04E4FF123CDAD2237D017C007F07CD
:10092000123D398F27E5277008FD7FFF123CB6D2B4
:1009300023302303126000C288C2A8C2AA758900AE
:1009400012373090633FE0B4FA06A3E064CE607BD8
:10095000E4F52774372527F582E43463F583E4F062
:100960000527E527B443EC90633F74FAF0A374CEF7
:10097000F0A374CCF0906345740AF0E4A3F0A304F0
:10098000F0A3F090633B74FFF0A3F0A3F0E4A3F0B6
:100990009063567403F0E4F527E5272401FFE43360
:1009A000FE74372527F582E43463F583E0FD123CBD
:1009B000920527E527C3944340DFE4F5A775A61EFB
:1009C00075A6E1907FF0F0A3F080FE90634A740377
:1009D000F0A374CCF0E4906349F090668CF0A3F03F
:1009E000123146C2B5123C47C21E123A1BD223C274
:1009F00025C2249065777408F09062B57424F0E401
:100A0000A3F090633FE09062B7F0906340E09062A3
:100A1000B8F0906341E09062B9F0906342E0906278
:100A2000BAF0906343E09062BBF0906344E0906260
:100A3000BCF0756801E4906578F0C21FC220C22145
:100A4000C222202318AF27FE7D03122F8AE4FF1253
:100A500032C87E0F7F5EE4FBFDFC122BA090668EF9
:100A6000E060037401F0E4906104F0F56A9065764B
:100A7000F0F56B123DBC75A70775A61E75A6E1D2F1
:100A8000AFC21BE4F56B906104E07003121DA190EE
:100A9000668FE06401701D9080007410F09080A853
:100AA00074FFF0A3F0A3F0A3F0E490668FF0D223DC
:100AB000C224C225908008E0F52730E405D21F74D7
:100AC00010F0E52730E508D2219080087420F0E589
:100AD0002730E608D2209080087440F0E56AC3947D
:100AE000034019908002E4F0908001F0908000F0C3
:100AF000E56A94064006E4F56A123A1B9080A0E08D
:100B000070031238289080B8E070031237AE9080DE
:100B1000D0E070031239BF908000E07013301F10D6
:100B2000122CA7906332EFF0D394004003120036EA
:100B3000908002E07006908000E06005D21D020AFD
:100B400083C21DE4F56A906104E06003020A832019
:100B50002312906579E0600C7E0F7F60122EA2E474
:100B6000906579F03021121227D2906332EFF0D3E2
:100B700094004005E0FF120032202003020D131202
:100B8000235B906332EFF07003020A83906376E098
:100B900054BF247F7003020C65147003020C3D24C3
:100BA000026003020CAC2023077E0F7F67122EA287
:100BB000906682E06003020D1390634EE070069031
:100BC0006352E06067906683E0FF90634EE0B50794
:100BD00024906684E0FE90634FE0B5061890668529
:100BE000E0FE906350E0B5060C906686E0FE9063F0
:100BF00051E06E6037906352E06F6003020D139016
:100C00006684E0FF906353E06F6003020D1390660B
:100C100085E0FF906354E06F6003020D13906686D9
:100C2000E0FF906355E06F6003020D13C21B9065F7
:100C3000787401F0123DF1756801020D1390668E13
:100C4000E060037401F090667BE0FF906378E06FF2
:100C50006003020D1390667BE004F0E4F568906594
:100C600076F0020D13301B03020D13906345E07004
:100C700003020A839062B4E06008906356741EF029
:100C800080069063567403F0123C6DD21BE4F56845
:100C9000906576F090668704F0E490667AF0A3F0B1
:100CA0002023707E0F7F75122EA2806790668EE0E3
:100CB00060037401F0301B52906376E020E74B90A4
:100CC0006378E0FF90667AE0FE6F600D906682E0E8
:100CD0007007EE146F703C801390667AE004F09019
:100CE0006332E0FFD394044003123A7590600074BD
:100CF00082F0A37401F0906378E0906002F07E606F
:100D00007F007D0312351B020A83201B0690668339
:100D100074FFF0201B03020E36E568706E123C155E
:100D2000EF60237E647F76906477E02404FD1235C3
:100D30001B906682E07009906356E0F568020A83B2
:100D4000E4F568020A83906687E0D3943C403C90C7
:100D50006682E070369062B4E0703090668704F08E
:100D6000123213E4906476F0A37412F090667BE084
:100D7000906478F0A374FDF090610563A201906423
:100D80007A63A2017F121220A98098123DE68F2774
:100D9000E527B401159060007483F0E4A3F07E6051
:100DA0007F007D0212351B020A83E527D3940140A0
:100DB0001C9060007483F0A37401F0E52724FEA367
:100DC000F07E607F007D0312351B020A83E56864B4
:100DD000016003020A83906576E004F02023077E19
:100DE0000F7F7F122EA2906576E0FFD39401400B17
:100DF000906356E0941E5003E004F0EFC394054066
:100E00000DC21BE4906578F0123DF1020A837C6606
:100E10007D8390634AE0FAA3E0FB7F021236AC7E4A
:100E2000647F76906477E02404FD12351B9063564E
:100E3000E0F568020A83E56864016003020A8390B2
:100E40006578E0146061147003020F3B14700302B4
:100E50000F4D24036003020A83E4F56A906682E082
:100E6000602D90634EE0FCA3E0FDA3E0FEA3E0FF55
:100E7000906683121C1D90634A7403F0A374CCF037
:100E800030B403020A839065787401F0020A8390FB
:100E900080027410F09065767401F07568129066A7
:100EA0008374FFF0020A83906683E0605D9064764D
:100EB0007480F09064787401F0E4A3F0A304F0A3CC
:100EC000743FF0A3747BF0E4F527747D2527F58249
:100ED000E43464F583747DF0747E2527F582E43470
:100EE00064F583E4F0E5272407906477F07C667D61
:100EF0008390634AE0FAA3E0FB7F021236AC7E6483
:100F00007F76E5272409FD12351B906682E060207C
:100F1000E4906578F0123C6DD21BE4F5689065763C
:100F2000F090668704F0E490667AF0A3F0020A83FA
:100F3000E4906578F0756812020A8390657874030E
:100F4000F0F568C2B57FFF123DDB020A83E49065CD
:0D0F500078F0123A1B756812020A8380FEC9
:010F5D002271
:10003600906377E0B444047F0180027F009063768A
:10004600E0B447047E0180027E00EE5F604A906362
:100056003FE0906378F0906340E0906379F09063BE
:1000660041E090637AF0906342E090637BF09063A6
:1000760043E090637CF0906344E090637DF090638E
:10008600777452F09062AE63A2019080A863A201D9
:100096007F061220A90208D6906332E0C394085066
:1000A600030208DF90633FE0FF906378E06F600330
:1000B6000208DF906340E0FF906379E06F6003021F
:1000C60008DF906341E0FF90637AE06F6003020807
:1000D600DF906342E0FF90637BE06F60030208DF1E
:1000E600906343E0FF90637CE06F60030208DF905B
:1000F6006344E0FF90637DE06F60030208DF906376
:1001060077E06444701A9080A8E0B4FF139062AE62
:1001160063A2019080A863A2017F061220A9801025
:100126009062B2E09080ACF09062B3E09080ADF067
:1001360090668EE060037401F090668F7464F090B0
:1001460063777452F0906376E0646D60030202791F
:100156007BFF7A0F798A1218367BFF7A0F79A49083
:10016600633FE0F530A3E0F531A3E0F532A3E0F517
:1001760033A3E0F534A3E0F5351218367530FF7574
:1001860031107532017533FF75341075350D7BFFEF
:100196007A0F79DA1218367BFF7A1079161218362A
:1001A6007BFF7A10797C1218367BFF7A1079A9903A
:1001B6006345E0F530A3E0F531A3E0F532A3E0F5C1
:1001C600331218367BFF7A1079D390633BE0F53013
:1001D600A3E0F531A3E0F532A3E0F5331218367B40
:1001E600FF7A1079F6906337E0F530A3E0F531A396
:1001F600E0F532A3E0F5331218367BFF7A11791356
:100206001218367BFF7A11793E90634EE0F530A3E3
:10021600E0F531A3E0F532A3E0F5331218367BFFA3
:100226007A11796C906352E0F530A3E0F531A3E0E2
:10023600F532A3E0F5331218367BFF7A11799A90DE
:100246006682E0F5301218367BFF7A1179C5906622
:100256008EE0F5301218367BFF7A1179F89062B489
:10026600E0F530121836122DAB7BFF7A12792A127E
:10027600183622906376E0644C70737E127F30FBF2
:10028600FDFC122BA090637EE0F528A3E0F529E49F
:10029600F52BE528906380F0A3E529F07E127F6BAD
:1002A6007C637D807B02122BA0E4F52A852982855A
:1002B6002883E0FF7480252AF582E43463F583EF12
:1002C600F00529E52970020528052AE52AB410DC7F
:1002D6007E127F6E7C637D807B10122BA0052BE542
:1002E6002BC3941040AC7E127F71122EA222906313
:1002F60076E0646C7060F52C7E127F73FBFDFC1259
:100306002BA0E4F52BE4906380F0A3E52CF07E129D
:100316007F6B7C637D807B02122BA0E4F52AA82CE0
:10032600E6FF7480252AF582E43463F583EFF00551
:100336002C052AE52AB410E67E127F6E7C637D804A
:100346007B10122BA0052BE52BC3940840B77E1219
:100356007F71122EA222906376E0644B7061F52ABB
:100366007468252AF582E43463F583E060327468A4
:10037600252AF582E43463F583E0F4602374682566
:100386002AF582E43463F583E0FF747E252AF5823C
:10039600E43463F583E0B50710052AE52AB408C0FE
:1003A6009061047432F00208D69063767421F030BE
:1003B60023030208D67E127FAE122EA20208D69022
:1003C6006376E0B4521A2023077E127FB6122EA25D
:1003D6009063767472F07E637F767D081234942281
:1003E600906376E0644970452023077E127FC11230
:1003F6002EA290637EE0F528A3E0F529E4F52A8590
:100406002982852883E0FF7480252AF582E43463F7
:10041600F583EFF00529E52970020528052AE52A66
:10042600B480DC7E637F767D8A1234942290637674
:10043600E0644370462023077E127FC9122EA290E5
:10044600637EE0F528A3E0F529E4F52A852982856F
:100456002883E493FF7480252AF582E43463F583C8
:10046600EFF00529E52970020528052AE52AB4805A
:10047600DB7E637F767D8A12349422906376E06415
:100486005A70532023077E127FD2122EA290637ECB
:10049600E0F528A3E0F5297C637D807B80AF29AE5B
:1004A60028123BE1E4F52A852982852883E493FF17
:1004B6007480252AF582E43463F583EFF00529E597
:1004C6002970020528052AE52AB480DB7E637F763B
:1004D6007D8A12349422906376E0644460030205B8
:1004E6006D90637EE0FF644470030208D6EFB4317A
:1004F6000CC2237E127FDE122EA20208D690637EE5
:10050600E0B4300CD2237E127FEA122EA20208D665
:1005160090637EE0B4320CD2247E127FF7122EA2B4
:100526000208D690637EE0B4330CC2247E137F05A6
:10053600122EA20208D690637EE0B4340CD2257E39
:10054600137F14122EA20208D690637EE0B4350CF7
:10055600C2257E137F21122EA20208D690637EE06A
:10056600FF123DA80208D6906104E070132023070D
:100576007E137F2F122EA29063767421F00208D686
:100586009061047432F0906376E0FFB45104C2AF18
:1005960080FEEF645770452023077E137F3D122EA1
:1005A600A290637FE0906332F0E4F52A906332E034
:1005B600FFE52AC39F40030208D67480252AF582E8
:1005C600E43463F583E0FF90637EE0252A24ADF5ED
:1005D60082E43461F583EFF0052A80D0906376E0FB
:1005E600645360030206902023077E137F48122E71
:1005F600A290633FE0FF9061B6E06F703C9063406D
:10060600E0FF9061B7E06F7030906341E0FF90616A
:10061600B8E0B50724906342E0FF9061B9E0B50702
:1006260018906343E0FF9061BAE0B5070C9063440D
:10063600E0FF9061BBE06F60169063767421F03046
:1006460023030208D67E137F57122EA20208D6E491
:10065600F52AE4F56BAF2AFE74AD252AF582E4345B
:1006660061F583E0FD123C92052AE52AC394FE401B
:10067600E1C2AFE4907FF0F0A3F0907FFD74AAF0A2
:10068600A374FFF0A37455F080FE906376E0644F88
:10069600705A90637EE0F528A3E0F529E529452800
:1006A600700A2023077E137F60122EA22023077E66
:1006B600137F67122EA2E4F52A7480252AF582E4B8
:1006C6003463F583E0852982852883F00529E529A9
:1006D60070020528052AE52AB480DE90668DE0249E
:1006E60080F090668CE03400F00208D6906376E0E5
:1006F6006445707490637EE0FEA3E0FF907FF0EEA9
:10070600F0A3EFF0D39400EE94044038907FF0E02D
:10071600FEA3E0FF90668CE0FCA3E0FD9FEC9E400C
:1007260023E42FFFEE3401FED3ED9FEC9E5015C25D
:10073600AF907FFD74AAF0A374FFF0A37455F0E4A4
:10074600F5A780FE7E137F69122EA27BFF7A1379AE
:1007560071907FF0E0F530A3E0F53190668CE0F51E
:1007660032A3E0F533121836906376E064656003D1
:100776000208DF90637EE0FFA3E0907FF0CFF0A356
:10078600EFF0E4F528F529D3907FF1E09529907FE5
:10079600F0E095284020E4F56B2529FFE528340193
:1007A600FE852982852883E0FD123C920529E529EC
:1007B6007002052880D17E137F7C1235A2EF4E6031
:1007C60020120003906345EFF0120003906346EF9A
:1007D600F0120003906347EFF0120003906348EFB6
:1007E600F07E137F821235A2EF4E60201200039036
:1007F600634EEFF012000390634FEFF01200039088
:100806006350EFF0120003906351EFF07E137F8880
:100816001235A2EF4E6020120003906352EFF012E1
:100826000003906353EFF0120003906354EFF0124D
:100836000003906355EFF07E137F8E1235A2EF4EC4
:10084600602012000390633BEFF012000390633CBC
:10085600EFF012000390633DEFF012000390633E49
:10086600EFF07E137F941235A2EF4E602012000344
:10087600906337EFF0120003906338EFF012000335
:10088600906339EFF012000390633AEFF0E4F52A33
:10089600E4F56BE52A2401FFE433FE7437252AF5D7
:1008A60082E43463F583E0FD123C92052AE52AC30F
:1008B600944340DCC2AFE4907FF0F0A3F0907FFD5C
:1008C60074AAF0A374FFF0A37455F0E4F5A780FEB4
:0908D6007E637F767D08123494E4
:0108DF0022F6
:103BA900AE07EEC39430400BEED394395005EE24A2
:103BB900D0FF22EEC39461400BEED394665005EE1C
:103BC90024A9FF22EEC39441400BEED3944650053D
:083BD900EE24C9FF22AF062211
:103D8E009062ADE004F070069062ACE004F09062D8
:0A3D9E00ACE0FEA3E0FF123D1C2282
:10000300123D8E123BA9EFC454F0FEC006123D8E82
:08001300123BA9D0E02FFF22EF
:10396200E4906A77F0123D8E906A78EFF0C394305B
:103972004018E0FFD394395011906A77E02405F59E
:1039820082E43461F583EFF08011906A77E02405D8
:10399200F582E43461F583E4F0800C906A77E00408
:1039A200F0E0D3940840BE752B00752C00752D00F5
:0C39B200E4F52E7B017A6179051221B743
:0139BE0022E6
:0435A2008E2D8F2EAD
:1035A6009062ACE4F0A374FFF0123D8EEF606EF40F
:1035B600606B852E82852D83E493B507EC752F010C
:1035C600E52E252FF582E4352DF583E493602590CD
:1035D60062ADE0252FFF9062ACE03400FE123D1C88
:1035E600E52E252FF582E4352DF583E493B5070402
:1035F600052F80CCE52E252FF582E4352DF583E4C5
:103606009370A6E52F24FFFFE434FFFE9062ADE041
:103616002FF09062ACE03EF07E007F0122E4FEFFD8
:013626002281
:103146007E137F9A1235A2EF4E70037F01227E1303
:103156007F9D1235A2EF4E600C123D8EEF24D0906B
:103166006682F08005E4906682F07E137FA31235B6
:10317600A2EF4E600C123D8EEF24D090668EF0804A
:1031860005E490668EF07E137FA91235A2EF4E609D
:103196000C123D8EEF24D024FF92198002C2197EB4
:1031A600137FAF1235A2EF4E600C123D8EEF24D086
:1031B6009062B4F08005E49062B4F090633F63A23D
:1031C6000190667C63A2017F061220A930193B7E1E
:1031D600137FB51235A2EF4E603012000390667C65
:1031E600EFF012000390667DEFF012000390667E0A
:1031F600EFF012000390667FEFF0120003906680F6
:0D320600EFF0120003906681EFF07F0022D0
:103B1C00906577E0C3947C40027F0A906577E0FE65
:103B2C0004F074B52EF582E43462F583EFF0BF0A2D
:103B3C0027906577E0FF04F074B52FF582E43462CA
:103B4C00F583E4F0906577E0FF1236279065777483
:093B5C0008F09062B6E004F022CA
:103A1B009080007480F090633763A201F583F58288
:103A2B0063A2017F081220A990633F63A2019080DB
:103A3B008863A2017F0A1220A99080927407F0A3D9
:103A4B0074D0F0A37406F0906349E0FF9080B1F05E
:103A5B009080E1EFF09080957455F0A3F09080008A
:0A3A6B007401F090800974F0F0225D
:10382800908009E04410F09080A0E070609080A142
:103838007482F09080A874FFF0A3F0A3F0A3F07F47
:10384800039080AEEFF0A374CBF09080007402F088
:10385800906ADF121C2900000000906ADFE0908067
:1038680040F0906AE0E0908041F0906AE1E090805A
:1038780042F0906AE2E0908043F0A3E4F0A3F0A362
:0D388800F0A3F0908018F0A3F0A3F0A3F0DF
:013895002210
:1039BF00908009E04440F09080D17482F07F0390B2
:1039CF0080DEEFF0A374CCF09080027402F0906A66
:1039DF00E3121C2900000000906AE3E0908058F089
:1039EF00906AE4E0908059F0906AE5E090805AF098
:1039FF00906AE6E090805BF0A3E4F0A3F0A3F0A35D
:0B3A0F00F0908030F0A3F0A3F0A3F0D3
:013A1A002289
:1037AE00908009E04420F09080B8E0706C9080B971
:1037BE007482F07F039080C6EFF07FCDA3EFF07F91
:1037CE00039080C4EFF0A374CDF09080C074FFF02E
:1037DE00A3F0A3F0A3F09080017402F0906AE712B8
:1037EE001C2900000000906AE7E090804CF0906A7F
:1037FE00E8E090804DF0906AE9E090804EF0906A9B
:10380E00EAE090804FF0A3E4F0A3F0A3F0A3F090D1
:09381E008024F0A3F0A3F0A3F054
:01382700227E
:1036AC008C288D29A907EAFDE975F018A424ACFF34
:1036BC00E5F034808F82F583EDF0EBFDE975F018C1
:1036CC00A4FFAEF024ACFBEE34808B82F583A3ED2B
:1036DC00F08529828C83E0FDEF24A8FFEE3480FE78
:1036EC008F82F583EDF08529828C83A3E08F828E07
:1036FC0083A3F0852982852883A3A3E0FDE975F0D7
:10370C0018A424A8FFE5F03480FE8F82F583A3A3D0
:10371C00EDF08529828C83A3A3A3E08F828E83A3F3
:04372C00A3A3F02241
:063494008D2DAB07AA0616
:10349A00908000E030E5079065797401F022906A27
:1034AA00DFE0FCA3E0FDA3E0FEA3E0F5318E308D62
:1034BA002F8C2EAE02AF038E838F8263A201E5307A
:1034CA00540744C0F58385318263A201AF2D1221CE
:1034DA001BE4FCFDFEE531252DF531EE3530F530E6
:1034EA00ED352FF52FEC352EF52E908040E52EF098
:1034FA00A3E52FF0A3E530F0A3E531F09080007446
:10350A0020F0AF31AE30AD2FAC2E906ADF121C1D09
:01351A00228E
:06351B008D28AB07AA0693
:10352100908002E030E5079065797403F022906A9B
:10353100E3E0FCA3E0FDA3E0FEA3E0F52C8E2B8DE0
:103541002A8C29AE02AF038E838F8263A201E52B01
:10355100540744D0F583852C8263A201AF28122140
:103561001BE4FCFDFEE52C2528F52CEE352BF52B77
:10357100ED352AF52AEC3529F529908058E529F011
:10358100A3E52AF0A3E52BF0A3E52CF090800274CB
:1035910020F0AF2CAE2BAD2AAC29906AE3121C1D92
:0135A1002207
:0232C8008F284D
:1032CA00908001E030E5099065797402F07F002270
:1032DA00906AE7E0FCA3E0FDA3E0FEA3E0F52C8EF4
:1032EA002B8D2A8C2990667C63A201E52B54074416
:1032FA00C8F583852C8263A2017F06122131E52C51
:10330A002406F52CE4352BF52BE4352AF52AE43589
:10331A0029F52990657A63A201E52B540744C8F57B
:10332A0083852C8263A201AF28122131E4FCFDFEC1
:10333A00E52C2528F52CEE352BF52BED352AF52A2B
:10334A00EC3529F52990804CE529F0A3E52AF0A36C
:10335A00E52BF0A3E52CF09080017420F0AF2CAEA1
:0D336A002BAD2AAC29906AE7121C1DAF287C
:013377002233
:102CA7009081E0E0F528052805280528052805284E
:102CB70005280528052805280528908010E0F52B0C
:102CC700A3E0F52CA3E0F52DA3E0F52E9081E1E03C
:102CD700F528052805280528052805280528052895
:102CE700052805280528908014E0F52FA3E0F53086
:102CF700A3E0F531A3E0F532E531B52D08E532B5AE
:102D07002E037F0022E4F528E531540744E0F583DC
:102D170085328263A20190637663A2017F08122144
:102D27006190637863A2019062AE63A2017F06128D
:102D370020A9906376E0F529A3E0F52AE4F5289029
:102D47006376E0702AA3E024F8F528E531540744B8
:102D5700E0F58385328274082582F582E43583F5B0
:102D67008363A20190637663A201AF28122161AE4B
:102D770029E4FCFDE532252AF532E5313EF531ED52
:102D87003530F530EC352FF52F908014E52FF0A373
:102D9700E530F0A3E531F0A3E532F0908000744010
:032DA700F0AF2862
:012DAA002206
:10235B009081E6E0F528052805280528052805289D
:10236B0005280528052805280528908028E0F52B49
:10237B00A3E0F52CA3E0F52DA3E0F52E9081E7E08B
:10238B00F5280528052805280528052805280528EA
:10239B0005280528052890802CE0F52FA3E0F530C3
:1023AB00A3E0F531A3E0F532E4F528E531B52D0ACC
:1023BB00E532B52E05C2200224C7E531540744F09F
:1023CB00F58385328263A20190637663A2017F0855
:1023DB00122161906376E0F529A3E0F52AE52A4501
:1023EB002970099080027410F07F0022906683E0C0
:1023FB00FFF46030906378E06F600302248E906688
:10240B0084E0FF906379E06F7079906685E0FF90D0
:10241B00637AE06F706D906686E0FF90637BE06F90
:10242B006031805F906378E0906683F0906379E031
:10243B00906684F090637AE0906685F090637BE021
:10244B00906686F090637CE0FFA3E090634ACFF048
:10245B00A3EFF0906376E0702AA3E024F8F528E56B
:10246B0031540744F0F58385328274082582F58256
:10247B00E43583F58363A20190637663A201AF28F1
:10248B00122161AE29E4FCFDE532252AF532E53156
:10249B003EF531ED3530F530EC352FF52FAF2EAE57
:1024AB002DAD2CAC2BAB32AA31A930A82FD3121CDB
:1024BB000C40099080027410F07F002290802CE574
:1024CB002FF0A3E530F0A3E531F0A3E532F09080D7
:0624DB00027440F0AF287E
:0124E10022D8
:1027D2009081E3E0F5280528052805280528052825
:1027E2000528052805280528052890801CE0F52BDA
:1027F200A3E0F52CA3E0F52DA3E0F52E9081E4E013
:10280200F52805280528052805280528052805286E
:10281200052805280528908020E0F52FA3E0F53053
:10282200A3E0F531A3E0F532E4F528E531B52D0A50
:10283200E532B52E05C221022928E531540744E8C4
:10284200F58385328263A20190600463A2017F0E48
:10285200122177906004E0F529A3E0F52A90600C3C
:10286200E0FFF4604A90667CE0FEEF6E7079A3E0D0
:10287200FF90600DE06F706F90667EE0FF90600EDB
:10288200E06F706390667FE0FF90600FE06F7057BB
:10289200906680E0FF906010E06F704B906681E080
:1028A200FF906011E06F703FE4906013F080089039
:1028B200601374FFF0D2D9906004E0702AA3E02480
:1028C200F2F528E531540744E8F583853282740E27
:1028D2002582F582E43583F58363A2019060046367
:1028E200A201AF28122177AE29E4FCFDE532252AA8
:1028F200F532E5313EF531ED3530F530EC352FF579
:102902002FAF2EAE2DAD2CAC2BAB32AA31A930A8F5
:102912002FD3121C0C5006E52A452970099080011C
:102922007410F07F0022908020E52FF0A3E530F0B4
:10293200A3E531F0A3E532F09080017440F0AF28B6
:012942002272
:042EA2008E2D8F2EB4
:102EA600908000E030E5079065797401F022906A21
:102EB600DFE0FCA3E0FDA3E0FEA3E0F5348E338D56
:102EC600328C31E534FFE5335407FEE42FF530EE5E
:102ED60034C0F52F853082F5837423F00530E53054
:102EE6007002052F532FC7F582852F83740AF005CC
:102EF60030E5307002052F532FC790633F63A20160
:102F0600852F8385308263A2017F0612211B7406FA
:102F16002530F530E4352FF52F852D83852E8263F8
:102F2600A201852F8385308263A2011220FFE4FC73
:102F3600FDFE906ADFE0F8A3E0F9A3E0FAA3E02F34
:102F4600FFEE3AFEED39FDEC38FCEF2408FFE43ED7
:102F5600FEE43DFDE43CFC906ADF121C1D906ADF36
:102F6600E0908040F0906AE0E0908041F0906AE165
:102F7600E0908042F0906AE2E0908043F09080001A
:032F86007420F0C4
:012F89002225
:0A2BA0008E2D8F2E8C2F8D308B317F
:102BAA00908000E030E5079065797401F022906A20
:102BBA00DFE0FCA3E0FDA3E0FEA3E0F5378E368D4F
:102BCA00358C34E537FFE5365407FEE42FF533EE4E
:102BDA0034C0F532853382F5837423F00533E53347
:102BEA00700205325332C7F582853283740AF005C2
:102BFA0033E533700205325332C790633F63A20153
:102C0A0085328385338263A2017F0612211B7406F3
:102C1A002533F533E43532F532852D83852E8263EB
:102C2A00A20185328385338263A2011220FF8F3885
:102C3A00EF2533F533E43532F532E5316017852F68
:102C4A008385308263A20185328385338263A20140
:102C5A00AF3112211BE53824082531F531FFE4FC98
:102C6A00FDFEE5372FF537EE3536F536ED3535F518
:102C7A0035EC3534F534908040E534F0A3E535F091
:102C8A00A3E536F0A3E537F09080007420F0AF3763
:0C2C9A00AE36AD35AC34906ADF121C1D64
:012CA600220B
:06306B008E288F298D2A3A
:10307100908000E030E5079065797401F022906A54
:10308100DFE0FCA3E0FDA3E0FEA3E0F5308E2F8D91
:103091002E8C2DE530FFE52F5407FEE42FF52CEEA5
:1030A10034C0F52B852C82F5837423F0052CE52C97
:1030B1007002052B532BC7F582852B83EBF0052C72
:1030C100E52C7002052B532BC790633F63A201854A
:1030D1002B83852C8263A2017F0612211B74062596
:1030E1002CF52CE4352BF52B85288385298263A2C9
:1030F10001852B83852C8263A201AF2A12211B74C7
:1031010008252AF52AFFE4FCFDFEE5302FF530EE17
:10311100352FF52FED352EF52EEC352DF52D908033
:1031210040E52DF0A3E52EF0A3E52FF0A3E530F067
:103131009080007420F0AF30AE2FAD2EAC2D906A90
:04314100DF121C1D60
:013145002267
:023627008F41D1
:10362900908000E030E5079065797401F022906A96
:10363900DFE0FCA3E0FDA3E0FEA3E0F5458E448DA9
:10364900438C42E545FFE5445407FEE42FFFEE3481
:10365900C09062B563A201F5838F8263A201AF4175
:1036690012211BE4FCFDFEE5452541F545EE3544F7
:10367900F544ED3543F543EC3542F542908040E59C
:1036890042F0A3E543F0A3E544F0A3E545F09080BB
:10369900007420F0AF45AE44AD43AC42906ADF12EE
:0236A9001C1DE6
:0136AB0022FC
:062F8A008E288F29AB0523
:102F9000908000E030E5079065797401F022906A36
:102FA000DFE0FCA3E0FDA3E0FEA3E0F52F8E2E8D75
:102FB0002D8C2CE52FFFE52E5407FEE42FF52BEE8C
:102FC00034C0F52A852B82F5837423F0052BE52B7D
:102FD0007002052A532AC7F582852A83EBF0052B58
:102FE000E52B7002052A90633F63A201852A838541
:102FF0002B8263A2017F0612211B7406252BF52B61
:10300000E4352AF52A532AC7E528852B82852A83A9
:10301000F0052BE52B7002052A532AC7F582852A75
:1030200083E529F0052BE52B7002052A532AC7E515
:103030002F240AF52FE4352EF52EE4352DF52DE459
:10304000352CF52C908040E52CF0A3E52DF0A3E580
:103050002EF0A3E52FF09080007420F0AF2FAE2E5D
:0A306000AD2DAC2C906ADF121C1D90
:01306A002243
:103D1C00A2AF9227C2AF438E2075D2028F828E83C0
:0C3D2C00E0FFE4F5D2538EDFA22792AF37
:013D38002268
:103C9200E5D220E0FBA2AF9227C2AF43D2028F82CD
:103CA2008E83EDF075D25063D250A22792AFE5D247
:033CB20020E0FB14
:013CB50022EC
:10373000E4FDED2401FFE433FE123D1C74372DF54A
:1037400082E43463F583EFF00DBD3FE6E4FDED2444
:103750007FFFE433FE123D1C742D2DF582E43461AD
:10376000F583EFF0742D2DF582E43461F583E0707C
:103770001B742D2DF582E43461F5837420F0742ED2
:103780002DF582E43461F583E4F080040DBD80BE44
:10379000E49061ACF0FDEDFF7E00123D1C74AD2D98
:0D37A000F582E43461F583EFF00DBDFEE924
:0137AD0022F9
:023BE1008B2D2A
:103BE300A2AF9227C2AF85A22E53A2FE8E838F82ED
:103BF30005A28C838D8274091221A5E52D53A2FEA3
:103C030043A2201221A753A2DF852EA2A22792AF9F
:013C1300FFB1
:013C1400228D
:103D3900A2AF9227C2AF8C838D82EF1221A543A235
:0C3D4900201221A753A2DFA22792AFFF97
:013D5500224B
:023CB6008F2855
:103CB800A2AF9227C2AFE4F5838D8274061221A5C4
:103CC800E52843A2201221A753A2DFA22792AF7FA3
:013CD80001EA
:013CD90022C8
:023CDA008F2831
:103CDC00A2AF9227C2AFE4F5838D82740A1221A59C
:103CEC00E52843A2201221A753A2DFA22792AF7F7F
:013CFC0001C6
:013CFD0022A4
:101FCE00A907E7FFA805EF93C3966008403B74FC92
:101FDE002FFF80F00F08EF93C3966008402B74FB21
:101FEE002FFF80E00F08EF93C3966008401B74FA32
:101FFE002FFF80D00F08EF93D3966008400B74F933
:10200E002FFF80C01F1F1F1F1FEF54FEF80303F783
:10201E00E893FC08E893FD08E893FE08E893FF2296
:10202E0009E993C39D6008402974FB29F980F109E1
:10203E00E993C39E6008401A74FA29F980E209E90F
:10204E0093D39F6008400B74F929F980D31919199D
:10205E001919E9C313C313FF22740093F8ECC39844
:10206E004024701F740193F8EDC3984019701474D6
:0E207E000293F8EEC398400E7009740393F8B5
:10208C00EFC39840037F00227F0122EDF8E6F008B1
:10209C00A3DFFA22EDF8E0F608A3DFFA22E0A3634F
:1020AC00A201F0A363A201DFF475A2002263A201D6
:1020BC00F0A363A20122E0A363A201F0A363A20137
:1020CC00E0A363A201F0A363A201E463A201F0A365
:1020DC0063A201DFE175A20022E0A363A2016DFE01
:1020EC00936CFDEE058393FC158363A201DFEA7507
:1020FC00A200227F00E493A363A201F00F600CA363
:10210C00E583C2E3F58363A20180EA75A20022E0B5
:10211C00A363A201F0A3E583C2E3F58363A201DF0D
:10212C00EE75A20022E0A363A201F0A3E583C2E452
:10213C00D2E3F58363A201DFEC75A20022E0A36376
:10214C00A201F0A3E58344F8C2E5F58363A201DFA5
:10215C00EC75A20022E583C2E3F583E0A363A20140
:10216C00F0A363A201DFEE75A20022E583C2E4D2E4
:0A217C00E3F583E0A363A201F0A3E2
:1021860063A201DFEC75A20022E58344F8F583E043
:10219600A363A201F0A363A201DFEE75A20022F9F8
:1021A60022C002C004C00612FFF0D006D004D0023E
:0121B6002206
:1013BB000A53656E643A20000A44617461206672B8
:1013CB006F6D207365727665723A000A4352432043
:1013DB006572726F722120000A53796E6320457219
:1013EB00726F722120000A526563204F4B2120003F
:1013FB003E2A2C312CCFE0F0E0ECE5F2F0FB20F1B3
:10140B00E8EDF5F0EEEDEDEEE3EE20EFEEF0F2E0D1
:10141B000A003E4C2C4230312C256C752CD1EAEE57
:10142B00F0EEF1F2FC20EEE1ECE5EDE02C35302CAA
:10143B003130302C3230302C3330302C3630302CA5
:10144B00313230302C323430302C343830300A00DA
:10145B003E422C4731302C2562752CC8EDE2E5F06D
:10146B00F1E8FF20EDE020EFF0E8B8ECE50A003EF4
:10147B00422C4731312C2562752CC8EDE2E5F0F199
:10148B00E8FF20EDE020EFE5F0E5E4E0F7E50A000A
:10149B003E422C4730322C2562752CD3EFF0E0E224
:1014AB00EBE5EDE8E520EFEEF2EEEAEEEC2020289E
:1014BB005254532D435453290A003E532C47303377
:1014CB002C256C752CC7E0E4E5F0E6EAE020F1F2A0
:1014DB00E0F0F2E020EFE5F0E5E4E0F7E828ECF1EE
:1014EB00290A003E2A2C312CC0E4E0EFF2E5F02073
:1014FB00F1E8EDF5F0EEEDEDEEE3EE20EAE0EDE0F8
:10150B00EBE02E20CFF0EEF2EEEAEEEB2022C3F072
:10151B00E0EDE8F2220A003E422C4731322C2562E4
:10152B00752CC7E0EFF0E5F220E3E5EDE5F0E0F632
:10153B00E8E820ECE5E0EDE4F0E00A003E422C4761
:10154B0031332C2562752CD0E5E6E8EC2022E2E560
:10155B00E4EEECFBE9220A003E422C4731342C2509
:10156B0062752C2B20ECE5E0EDE4F020EFE5F0E5E7
:10157B00E420EEF2EAF0FBE2E0FEF9E8EC20F4EB1B
:10158B00E0E3EEEC0A003C21003C4230313D003CF4
:10159B004731303D003C4731313D003C4730323D17
:1015AB00003C4730333D003C4731323D003C473136
:1015BB00333D003C4731343D000008040C020A0661
:1015CB000E0109050D030B070F001123324657655A
:1015DB00748C9DAFBECADBE9F810013322564775F8
:1015EB00649C8DBFAEDACBF9E821300213677644E9
:1015FB0055ADBC8E9FEBFAC8D931201203776654D8
:10160B0045BDAC9E8FFBEAD8C942536170041527C8
:10161B0036CEDFEDFC8899ABBA52437160140537B7
:10162B0026DECFFDEC9889BBAA63724051253406A8
:10163B0017EFFECCDDA9B88A9B7362504135241697
:10164B0007FFEEDCCDB9A89A8B8495A7B6C2D3E180
:10165B00F008192B3A4E5F6D7C9485B7A6D2C3F177
:10166B00E018093B2A5E4F7D6CA5B48697E3F2C068
:10167B00D129380A1B6F7E4C5DB5A49687F3E2D057
:10168B00C139281A0B7F6E5C4DC6D7E5F48091A348
:10169B00B24A5B69780C1D2F3ED6C7F5E49081B337
:1016AB00A25A4B79681C0D3F2EE7F6C4D5A1B08228
:1016BB00936B7A48592D3C0E1FF7E6D4C5B1A09217
:1016CB00837B6A58493D2C1E0F0089129B24AD3633
:1016DB00BF48C15AD36CE57EF78108931AA52CB786
:1016EB003EC940DB52ED64FF76028B109926AF3476
:1016FB00BD4AC358D16EE77CF5830A9118A72EB566
:10170B003CCB42D950EF66FD74048D169F20A93255
:10171B00BB4CC55ED768E17AF3850C971EA128B345
:10172B003ACD44DF56E960FB72068F149D22AB3035
:10173B00B94EC75CD56AE378F1870E951CA32AB125
:10174B0038CF46DD54EB62F97008811A932CA53E15
:10175B00B740C952DB64ED76FF89009B12AD24BF05
:10176B0036C148D35AE56CF77E0A8318912EA73CF5
:10177B00B542CB50D966EF74FD8B029910AF26BDE5
:10178B0034C34AD158E76EF57C0C851E9728A13AD5
:10179B00B344CD56DF60E972FB8D049F16A920BBC5
:1017AB0032C54CD75EE168F37A0E871C952AA338B5
:1017BB00B146CF54DD62EB70F98F069D14AB22B9A5
:0917CB0030C74ED55CE36AF178E9
:103D5C00526690000000000000000000000000000F
:053D6C00000000000052
:103CFE00906A6CE06FFC9016D493FE906A6BE06E47
:0D3D0E00A3F0AF04EF9015D493906A6BF012
:013D1B002285
:0100320022AB
:10001E00EF540F9015C493FEC454F0FEEFC4540F6A
:04002E00932EFF22EC
:103C150030162CE4906476F0E51C24FEFFA3F090AA
:103C2500667BE0906478F0A37408F090696B63A2FA
:103C35000190647A63A2011220A9C2167F01227F36
:023C450000225B
:103AC900C227E4FEE51B64056032BF7E07D205E428
:103AD900F517F51BEF30E707431001051B80065367
:103AE90010FEE4F51B0517E517B4080885101FD269
:103AF90027E4F517E51025E0F510800CEF30E70510
:103B0900D205A22722E4F51BEF25E0FF0EBE08B47B
:023B1900A227E1
:013B1B002287
:10389600E4FEE51625E0F516EF30E736431601207F
:1038A60027330515E515B4052CE4F515051AE51AB3
:1038B600B408170514E514AC137002051314F58249
:1038C6008C83E516F0051DE4F51AE51625E0F516D8
:1038D6008003E4F515051AE51AB408170514E5146E
:1038E600AC137002051314F5828C83E516F0051DE2
:0D38F600E4F51AEF25E0FF0EEE6408709572
:0139030022A1
:103C4700906A7174FFF0A374B8F0E4906A70F09012
:103C57006A6F04F0E4906A6DF012266012390490DE
:063C670066A27401F022C8
:103C6D0075657E7562A0C208D210C216D230C2141C
:103C7D00C202C215D201C212E4F561F55CD290D236
:053C8D0091123DCC2264
:042A95008E298F2ACD
:102A9900906A6BE0906A75F0906A6CE0906A76F0E3
:102AA900E4F51DF515906A6BF0A3F0AB2AAA297518
:102AB90013697514EB301125851482851383740A03
:102AC900F00514E51470020513F58285138374AAC1
:102AD900F00514E51470020513051D051D85148202
:102AE900851383747EF00514E51470020513051D22
:102AF900E4F51A906A73F0906A73E0C39D50498BAC
:102B0900828A83E0FF12001E906A74EFF0906A6C6B
:102B1900E06F906A74F0E0FF9016D493FE906A6BB0
:102B2900E06EA3F0EF9015D493906A6BF00BEBAEC7
:102B39000270010A14F5828E83E0FFC227123896CB
:102B4900906A73E004F080AF906A6CE0FF12001E97
:102B5900C227123896906A6BE0FF12001EC2271234
:102B69003896D2277F7E123896D227E4FF123896FC
:102B7900D2027C697DEB8C138D143025097E137F7D
:102B8900BBAB1D122BA0906A75E0906A6BF0906A3E
:062B990076E0906A6CF08A
:012B9F002213
:103A75008F2820022130120E7E697F2BE52824FC39
:103A8500FD122A95800C7E637F7AE52824FCFD12C1
:103A95002A95C212801C201219852819D21290630A
:103AA5007A63A20190692B63A201E52824FCFF1229
:103AB50020A930250B7E137FC3E4FBFDFC122BA050
:043AC5008528282206
:10321300E4FF0F2405F582E43461F5837408F00FAD
:1032230074052401F582E43461F583E4F07C667D62
:1032330095FEED1DAA0470011CF5828A83E0FBAAAA
:10324300070F74052AF582E43461F583EBF00EBEB3
:1032530004E07C667D99E4FEED1DAA0470011CF573
:10326300828A83E0FBAA070F74052AF582E434619E
:10327300F583EBF00EBE04E07C667D9DE4FEED1D60
:10328300AA0470011CF5828A83E0FBAA070F740568
:103293002AF582E43461F583EBF00EBE04E07C662C
:1032A3007DA1E4FEED1DAA0470011CF5828A83E072
:1032B300FBAA070F74052AF582E43461F583EBF06A
:0432C3000EBE04E057
:0132C70022E4
:103D7200D201D291D208E4F51CF51B906A6CF09046
:0C3D82006A6BF0F51775116975126B2261
:10294300200803022A5DE5605438655B7003022AA0
:1029530094E55B24085438F55B131313541F244B7D
:10296300F8E6F51820053020072DFF123AC950D696
:10297300AF1F12001E123CFE0512E512AE117002CB
:10298300051114F5828E83E51FF0051CE51CD39415
:102993004040B3D20780AFE51CD394024005200723
:1029A30002D216C208C205E4F549D230C291906A38
:1029B3006CE0FF906A6BE04F6047C21630250D7ED6
:1029C300137FD67C697D6BAB1C122BA090669AE0BB
:1029D300FCA3E0FDA3E0FEA3E0FFE4FAF9F8EF2493
:1029E30001FFEA3EFEE93DFDE83CFC90669A121CBD
:1029F3001D90696BE0705E20075BC230123D7280F0
:102A03005490696BE07014C2163025497E137FE33E
:102A13007C697D6BAB1C122BA0803A30250D7E1395
:102A23007FF17C697D6BAB1C122BA0906692E0FC5E
:102A3300A3E0FDA3E0FEA3E0FFE4FAF9F8EF24012D
:102A4300FFEA3EFEE93DFDE83CFC906692121C1D48
:102A5300E4906A6EF0C207022949203034E54BB492
:102A63007E0F300308E4F549D230C20322123D72CF
:102A730022E54BB56216200613D2019066A4E0FF4F
:102A8300A3E0906929CFF0A3EFF0C209E4F549D29E
:022A93003022EF
:101DA1009066A2E0B4010630B403021FCDE4906650
:101DB100A2F0300F2DC3E5489564FFE5479563FE1A
:101DC100D3EF9440EE940040197B087D40AF64AEA0
:101DD1006312306BE5642440FFE43563540FF5630F
:101DE1008F64201B05D291D29022301A2630B4087C
:101DF100906828E004F080069068287401F09068EB
:101E010028E0C39414400280FEC21A9067A6E060E5
:101E11000214F0301003122943301476E561655C39
:101E2100603BE56124085438FFE55C54386F70036A
:101E3100021FCDE51D7003021FCD0514E514AC137F
:101E41007002051314F5828C83E0FEE56113131310
:101E5100541F2453F8A6068F61151D80C5C290C278
:101E610014C202906696E0FCA3E0FDA3E0FEA3E0AD
:101E7100FFE4FAF9F8EF2401FFEA3EFEE93DFDE84F
:101E81003CFC906696121C1DD215D2B1E49067A657
:101E9100F022300803021FCD300253E561655C601A
:101EA10003021FC330B10AC2B19066A3E09067A6D6
:101EB100F030130C30B0099067A6E06003021FCD2B
:101EC1000514E514AE137002051314F5828E83E038
:101ED100FFE561131313541F2453F8A607E561248A
:101EE100085438F561151DD214D290021FC3301267
:101EF10006AF19123A7522E561655C6003021FC3E2
:101F0100300403021FC330B10AC2B19066A3E0904E
:101F110067A6F030130C30B0099067A6E0600302A9
:101F21001FCD20012590669EE0FCA3E0FDA3E0FE0D
:101F3100A3E0FFE4FAF9F8EF2401FFEA3EFEE93DF0
:101F4100FDE83CFC90669E121C1DC201E561131365
:101F510013541F2453F8760AE56124085438F561B7
:101F6100131313541F2453F876AAE5612408543837
:101F7100F561131313541F2453F8E4F6E5612408A3
:101F81005438F561131313541F2453F8E4F6E56133
:101F910024085438F561131313541F2453F8E4F63D
:101FA100E56124085438F561131313541F2453F8C1
:101FB100E4F6E56124085438F561E55C24105438F1
:0D1FC100F51EE51EB55C05751E40D2B1226F
:0B3DE600301505C2157F01227F00226E
:102DAB00906A70E06022A3E0FEA3E0FFC3E49FFF04
:102DBB00E49EFEAB07FA3395E0F9F87F007EC27D07
:102DCB00017C00123B658021906A71E0FEA3E0FF5D
:102DDB00C3E49FFFE49EFEAB07FA3395E0F9F8E4FA
:102DEB007F207E1CFDFC123B65906A73121C1D7BC1
:102DFB00FF7A1379FB1218367BFF7A14791D906AD0
:102E0B0073E0FCA3E0FDA3E0FEA3E0F5338E328D6F
:102E1B00318C301218367BFF7A14795BA20EE433B7
:102E2B00F5301218367BFF7A14797AA20BE433F55E
:102E3B00301218367BFF7A14799BA213E433F530EA
:102E4B001218367BFF7A1479C59066A3E075F00AE9
:102E5B00A4FFAEF0E48F338E32F531F53012183615
:102E6B007BFF7A1479EE1218367BFF7A157922A242
:102E7B0004E433F5301218367BFF7A157947A21725
:102E8B00E433F5301218367BFF7A157963A211E41F
:062E9B0033F53012183679
:012EA100220E
:102660007E157F911235A2EF4E70037F01227E15F9
:102670007F941235A2EF4E70030227071239629041
:102680006A73121C1DE4FFFEFDFC906A73E0F8A360
:10269000E0F9A3E0FAA3E0FBC3121C0C6025906AEA
:1026A00073E0F8A3E0A3E0A3E0E47F207E1CFDFC40
:1026B000121B6C121BFE906A71EEF0A3EFF0E49017
:1026C0006A70F0E47FB07E04FDFC906A73E0F8A3CA
:1026D000E0F9A3E0FAA3E0FBD3121C0C4038906AA7
:1026E000707401F0906A73E0F8A3E0A3E0A3E07FC8
:1026F000007EC27D017C00121B6C121BFE906A7171
:10270000EEF0A3EFF0800F906A7174FFF0A374B83D
:10271000F0E4906A70F07E157F9A1235A2EF4E6059
:102720000C123D8EEF24D024FF920E8002C20E7E4A
:10273000157FA01235A2EF4E600C123D8EEF24D013
:1027400024FF920B8002C20B7E157FA61235A2EFEA
:102750004E600C123D8EEF24D024FF92138002C2F3
:10276000137E157FAC1235A2EF4E6013123962E46E
:102770007B0AFAF9F8121B6C9066A3EFF08005E46F
:102780009066A3F07E157FB21235A2EF4E600C1258
:102790003D8EEF24D024FF92048002C2047E157F78
:1027A000B81235A2EF4E600C123D8EEF24D024FFFC
:1027B00092178002C2177E157FBE1235A2EF4E60BF
:1027C0000C123D8EEF24D024FF92118002C2117FA3
:0127D0000008
:0127D10022E5
:033DF100C2AE223D
:103DA800BF360BD20FE4F547F548F563F564BF3726
:043DB80002C20F2212
:10390400C2A9438902906A72E0FFF58C8F8A75D947
:103914000475DA4875DB3175DC4975DD4975DE31CE
:10392400E4F5E9F5F9F5EBF5FB906A70E0601675DE
:10393400EC1075ED10E4F5FCF5FD755F08755D1090
:10394400755E01801375EC8075ED80E4F5FCF5FD82
:0E395400755F80F55D755E10E4F5EEF5FE2200
:0E3DCC00E4FFD28C75D84075B740D2AED2AFAE
:013DDA0022C6
:030033000224E2C2
:0B24E200C0E0C083C082C0D075D008ED
:1024ED00C2AF30DC56C3E5EC95EEC3955F5012E5F7
:1024FD005E25ECF5EC30D70405FC801685FCFC80E0
:10250D0011C3E5EC955EF5EC30D70415FC80038521
:10251D00FCFC300F24854882854783E590F0054803
:10252D00E54870020547F582854783E5EEF00548DD
:10253D00E5487002054753470FC2DC30D929300FEB
:10254D0024854882854783E590F00548E54870026B
:10255D000547F582854783E5EBF00548E5487002B0
:10256D00054753470FC2D930DA6AE55D700405FCA3
:10257D008010E55D25ECF5EC30D70405FC80038576
:10258D00FCFC30104DE5495480F546E54925E0F554
:10259D00493097020549200E03634901303019E592
:1025AD004965656006E54965627027755B00756074
:1025BD000085494BC230801A0560E56054077012E2
:1025CD0053603FE560131313541F244BF8A6497550
:1025DD004900C2DA30DB71E55D700405FD8010E560
:1025ED005D25EDF5ED30D70405FD800385FDFDE599
:1025FD0061655C6029E55C54077013E55C1313138A
:10260D00541F2453F8E6F54A200B03634AFFE54AAD
:10261D00339296E54A25E0F54A055C535C3FB2924C
:10262D00300F23854882854783E590F00548E548BE
:10263D0070020547F582854783E4F00548E548704B
:0A264D0002054753470FC2DBD2AF6E
:09265700D0D0D082D083D0E03253
:103414000208E0E493A3F8E493A34003F68001F2E6
:1034240008DFF48029E493A3F85407240CC8C333B9
:10343400C4540F4420C8834004F456800146F6DF88
:10344400E4800B0102040810204080903D56E47E85
:10345400019360BCA3FF543F30E509541FFEE4937D
:10346400A360010ECF54C025E060A840B8E493A344
:10347400FAE493A3F8E493A3C8C582C8CAC583CA6F
:10348400F0A3C8C582C8CAC583CADFE9DEE780BE27
:013D71000051
:101B300075F008758200EF2FFFEE33FECD33CDCC6C
:101B400033CCC58233C5829BED9AEC99E5829840EF
:101B50000CF582EE9BFEED9AFDEC99FC0FD5F0D6CC
:101B6000E4CEFBE4CDFAE4CCF9A88222B800C1B9F6
:101B70000059BA002DEC8BF084CFCECDFCE5F0CB34
:101B8000F97818EF2FFFEE33FEED33FDEC33FCEB6D
:101B900033FB10D703994004EB99FB0FD8E5E4F928
:101BA000FA227818EF2FFFEE33FEED33FDEC33FC15
:101BB000C933C910D7059BE99A4007EC9BFCE99A09
:101BC000F90FD8E0E4C9FAE4CCFB2275F010EF2F4E
:101BD000FFEE33FEED33FDCC33CCC833C810D7074E
:101BE0009BEC9AE899400AED9BFDEC9AFCE899F889
:0E1BF0000FD5F0DAE4CDFBE4CCFAE4C8F9221C
:103B6500C2D5E830E70FB2D5E4C39BFBE49AFAE48B
:103B750099F9E498F8EC30E717B2D5123B9B121B84
:103B85006CE4C39BFBE49AFAE499F9E498F88003A2
:103B9500121B6C30D50DE4C39FFFE49EFEE49DFD32
:043BA500E49CFC227E
:0E1BFE00C3E49FFFE49EFEE49DFDE49CFC22F8
:101C0C00EB9FF5F0EA9E42F0E99D42F0E89C45F02E
:011C1C0022A5
:0C1C1D00ECF0A3EDF0A3EEF0A3EFF0223A
:101C2900A8828583F0D083D082121C40121C4012F6
:101C39001C40121C40E473E493A3C583C5F0C5831B
:101C4900C8C582C8F0A3C583C5F0C583C8C582C805
:011C59002268
:1017D400E53C2430F8E6053C22782D302E027830A2
:1017E400E475F001121D01021C5A2027EB7F2ED252
:1017F400278018EF540F2490D43440D4FF302B0B9F
:10180400EF24BFB41A0050032461FFE53D600215C4
:101814003D0540E5407002053F302E0D782DE475FE
:10182400F001121D01EF021CA0023B1C7403D22E16
:101834008003E4C22EF53C8B2D8A2E892FE4F53DDE
:10184400F53FF540E53D60077F2012180F80F575E0
:101854003EFFC228C227C229C22AC22CC22DC22FCF
:101864001217DDFF700D302E057F00121820AF40D7
:10187400AE3F22B4255FC2D5C22B1217DDFF24D0A0
:10188400B40A00501A75F00A783D30D50508B6FF41
:101894000106C6A426F620D5047002D22A80D924D3
:1018A400CFB41A00EF5004C2E5D22B021A20D2287A
:1018B40080C6D22780C0D22980BCD2D580BAD22C8F
:1018C40080B47F2012180F2029077401B53D004011
:1018D400F11217D4FF12180F021848D22FD22D80FC
:1018E400951217D4FB1217D4FA1217D4F94A4B7075
:1018F4000679F17A1A7BFF20292EE53D602A7E00C5
:101904008E82758300121C7360060EEE653E70F0C5
:10191400C2D5EBC0E0EAC0E0E9C0E0EE121A67D03D
:10192400E0F9D0E0FAD0E0FB121C5AFF60AAEBC049
:10193400E0EAC0E0E9C0E012180FD0E02401F9D0D9
:10194400E03400FAD0E0FBE53E0460DCD53ED9800B
:10195400877BFF7A1A7963D229809C791080027977
:1019640008C22DC22F8008D2D5790A8004790AC210
:10197400D5E53E047002F53EE4FAFDFEFF1217D4ED
:10198400FC7B082028131217D4FD7B1030270A1281
:1019940017D4FE1217D4FF7B20EC3382D592D55096
:1019A40013C3E43027069FFFE49EFEE42028039D32
:1019B400FDE49CFCE4CBF8C228EC700CCFCECDCC7B
:1019C400E824F8F870F38017C3EF33FFEE33FEED2D
:1019D40033FDEC33FCEB33FB994002FB0FD8E9EB0E
:1019E400302805F8D0E0C448B228C0E00AEC4D4ED7
:1019F4004F78207B0070C2EAB53E0040BCC0E012C4
:101A04001A69D0F0D0E0202804C4C0E0C4B228C0D1
:101A1400F01217F8D0F0D5F0EB021848121D601838
:101A2400E553195F5818B64C18B24219634F196B35
:0F1A340044196B4918CB4319715519554619556B
:101A4300451955471B115018BA2D18BE2E18E12BF6
:101A530018C22318DF201AFA2A187A48000018D966
:101A63003F3F3F00790AA2D5202A14302C09B91030
:101A7300020404B9080104A2D5202D025001042058
:101A830029689229B53D005034C0E07F20302A19DF
:101A93007F30A229722D722C500F121AC0C229C294
:101AA3002DC22CC22F7F30800F302C03E9C0E012EF
:101AB300180F302C03D0E0F9D0E0B53DCC302C1713
:101AC3007F30B9100C12180F7F58302B077F7880A6
:101AD30003B9080312180F3029057F2D02180F7F51
:101AE30020202FF87F2B202DF322922980CF286EE0
:101AF300756C6C2900D2281217D43028F8C22878C4
:101B03003D30D50108F602187A2D50434958121773
:101B1300D42403B405004001E4901B0C9312180075
:0D1B2300743A121800D22A753D0402195FB1
:1021B7008B288A29892AE4F534F533F532F531F588
:1021C7002FF530E52C452D452B6012EBC0E0EAC01A
:1021D700E0E9C0E0AB2BAA2CA92D121D11AB2805F5
:1021E7002AE52AAA297002052914F9121C5AF5357D
:1021F700C394094007E535D3940D40E1E5356420E4
:1022070060DBE535B42D054330038016E535B42B87
:1022170005433001800C74FF252AF52A74FF352900
:10222700F529E52E60046410703FAB28AA29A92A76
:10223700121C5A64306009E52E702E752E0A80290B
:10224700900001121C73FF64786004EFB4581343C5
:102257003001752E107402252AF52AE43529F5294F
:102267008007E52E7003752E08AB28052AE52AAAF4
:10227700297002052914F9121C5AF535C3946140D7
:102287000AE535D3947A50035335DF74D02535F5F5
:1022970035C3940A400CE5359411406D74F9253522
:1022A700F535E535D3952E506043300185343985B2
:1022B7003338853237853136AF2E7E00E4FCFDABEF
:1022C70034AA33A932A831121CB2C8ECC8C9EDC967
:1022D700CAEECACBEFCBE4FCFDFEEB2535F534EEB9
:1022E7003AF533ED39F532EC38F531AF34AE33AD7D
:1022F70032FCAB39AA38A937A836D3121C0C5003C5
:10230700022270433004022270E53020E003E480AB
:102317002DE52C452D452B601EAB28E52A24FFF91A
:10232700E52934FFFAEBC0E0EAC0E0E9C0E0AB2BF7
:10233700AA2CA92D121D11E53030E20774FFFFFE0C
:10234700FDFC22E530AF34AE33AD32AC3130E103C2
:04235700021BFE2245
:101C5A00BB010689828A83E0225002E722BBFE0288
:091C6A00E32289828A83E49322BB
:101C7300BB010CE58229F582E5833AF583E0225026
:101C830006E92582F8E622BBFE06E92582F8E22270
:0D1C9300E58229F582E5833AF583E493228A
:101CA000BB010689828A83F0225002F722BBFE0123
:021CB000F3221D
:101CB200E88FF0A4CC8BF0A42CFCE98EF0A42CFCD1
:101CC2008AF0EDA42CFCEA8EF0A4CDA8F08BF0A44F
:101CD2002DCC3825F0FDE98FF0A42CCD35F0FCEBAE
:101CE2008EF0A4FEA9F0EB8FF0A4CFC5F02ECD3973
:0F1CF200FEE43CFCEAA42DCE35F0FDE43CFC22E0
:101D0100FAE6FB0808E6F925F0F618E6CA3AF622E3
:101D1100BB011A89828A83D0F0D0E0F8D0E0F9D0F3
:101D2100E0FAD0E0FBE8C0E0C0F0021D8F5016E9F8
:101D3100F8D083D082D0E0F9D0E0FAD0E0FBC082C5
:101D4100C083021D86BBFE16E9F8D083D082D0E0A5
:0F1D5100F9D0E0FAD0E0FBC082C083021D9822D7
:101D6000D083D082F8E4937012740193700DA3A312
:101D700093F8740193F5828883E473740293686026
:061D8000EFA3A3A380DF26
:091D8600EBF608EAF608E9F62282
:091D8F00EBF0A3EAF0A3E9F02255
:091D9800EBF208EAF208E9F2227C
:00000001FF
